:100000000C945D000C94C9010C947A000C947A0055
:100010000C947A000C947A000C947A000C947A0078
:100020000C947A000C947A000C947A000C947A0068
:100030000C947A000C947A000C947A000C947A0058
:100040000C947A000C947A000C947A000C947A0048
:100050000C947A000C947A000C947A000C947A0038
:100060000C947A000C947A0009021200010100A09D
:10007000FA09040000000000000012011001FF0056
:100080000008C016DC050401010200010E03550042
:10009000530042006100730070001C03770077007A
:1000A00077002E00660069007300630068006C0032
:1000B0002E00640065000403090411241FBECFEF65
:1000C000D8E0DEBFCDBF11E0A0E0B1E0E0E7F1E1B4
:1000D00002C005900D92A230B107D9F721E0A2E04D
:1000E000B1E001C01D92AA34B207E1F70E94A40852
:1000F0000C94B6080C940000CF93DF936091280114
:10010000635067FD14C0209125018CE090E0821BB4
:100110009109EC01C45DDE4F809124018D3209F418
:1001200050C08091020187FD91C0109228018091FA
:10013000010184FF39C0C0910001CF3FA9F1C9304E
:1001400008F467C0C850C09300018091180198E876
:10015000892780931801C8E08091020187FDA0C023
:10016000209126013091270186FF67C0A9E1B1E007
:10017000F9018C2F94919D9331968150D9F78FEF8F
:100180008C0F90E00196280F391F309327012093A0
:1001900026016C2F89E191E00E94C501CC5FCC3033
:1001A00009F047C0C093010194E189B1847831F42A
:1001B0009150D9F71092290110922301DF91CF912C
:1001C0000895683009F0B1CF83EC809318018AE577
:1001D00080930101109202018881807609F041C06C
:1001E0002A81109221019981911147C01092220118
:1001F00021E231E082E030932701209326019F81A4
:10020000911104C09E81981708F4892F80930001F2
:100210008CCF109200018091180198E88927809373
:100220001801C11199CF60E089E191E00E94C501F8
:10023000C4E09FEF90930001B5CFD901E9E1F1E06F
:100240008C2F9D9191938150E1F799CFCE010E941F
:10025000D1078F3F09F1882309F467CF109200017D
:1002600064CFCE010E94B8058F3F49F6988197FD73
:100270002CC090E890930201C9CF953009F19630D7
:1002800031F1983079F1993089F181E09A3009F0B3
:1002900080E021E231E0AFCF8EE18093010145CFD4
:1002A0006C2F89E191E00E945207C82F893008F431
:1002B00070CF8FEF80930001CEE1C093010174CF26
:1002C0002093290121E231E096CF8E81D2CF9B810C
:1002D0009130C9F0923079F09330E9F090E4909346
:1002E00002018DCF2BE231E081E085CF20932B01FD
:1002F00021E231E080CF88E690E09093270180935F
:10030000260182E1EBCF8AE790E09093270180936A
:10031000260182E1E3CF211108C086EB90E09093A3
:1003200027018093260184E0D9CF213051F022307B
:10033000A9F68CE890E090932701809326018EE047
:10034000CDCF8AE990E090932701809326018CE13C
:10035000C5CFE9E6F0E0808183608083E89A089564
:10036000A82FB92F80E090E041E050EA609530E09E
:1003700009C02D9182279795879510F0842795279E
:10038000305EC8F36F5FA8F30895EADF8D939D9305
:100390000895CF93CFB7CF93DF93C3954F9BE9F7E2
:1003A0004F9B0BC04F9B09C04F9B07C04F9B05C085
:1003B0004F9B03C04F9B01C089C06F93C091250123
:1003C000DD27C45DDE4F2F9365E54F9B03C02F9162
:1003D0006F91E6CF0F931F934F9320E040E15F931F
:1003E00009B1047807FB27F93F9350E03BE039C09F
:1003F000147840642F77012F5F5F1EC0406819B1E9
:1004000014782F7752501FC0406409B12F770478B9
:10041000D1F15F5F00C023C0406219B12F7714781B
:1004200091F15F5F00C025C004781027515012F48D
:100430005D5F0000115027952C3F19B1C8F6147864
:100440000127015027952C3FC8F64227499309B14F
:10045000047810274F73115027952C3FA8F6469526
:10046000469519B1147879F00127015027952C3F52
:1004700098F66B5A60F3315009B1B0F600C011E044
:100480001CBB002717C03B503195C31BD04011E067
:100490001CBB0881033CF9F00B34E9F020912301E7
:1004A0001981110F1213EDCF093651F10D3211F0F0
:1004B000013E39F700932A013F915F914F911F91BF
:1004C0000F912F916F91CCB3C0FD67CFDF91CF918A
:1004D000CFBFCF91189520912A01222369F3109163
:1004E0002801112339F534303AF130932801209353
:1004F0002401109125013BE0311B309325011CC0E4
:10050000009128010130B4F40AE53091010134FD75
:1005100014C000930101C8E1D1E013C0052710E029
:1005200000C000000BB91AC0052710E0221F1DC033
:1005300010E021C04AE502C032ED432FC4E1D0E013
:1005400032E01AB114685F9A0BB11AB954E820E886
:1005500065E320FF05270BB9279517951C3FF0F69B
:100560006695B8F7B1F720FF05270BB927951795C2
:100570001C3FD0F62795179517FF052700001C3F55
:100580000BB9B0F629913A9519F70B77109129011B
:10059000110FC651D0400BB911F01093230111E097
:1005A0001CBB00681AB11B77402F4B7754E05A955B
:1005B000F1F70BB91AB94BB97FCF582F48E080E05B
:1005C00057FD18C02B98550F880F1C998F5F2D9AD7
:1005D00036B52091470196B5931B9217E0F32D98FD
:1005E00036B52091470196B5931B9217E0F3415021
:1005F00039F708952B9AE7CF8EBD0DB407FEFDCFD6
:100600008EB50895DC01CB0121E1B695A7959795AC
:1006100087952A95D1F7209146012817D9F0809324
:100620004601E0914301F09144018DE40995E09188
:100630004301F091440180E00995E0914301F0917C
:100640004401809146010995E0914301F0914401F4
:1006500080E009940895809145018CBD809142010C
:100660008DBD08958823A1F08830D0F52DED32E0BE
:1006700030934401209343018430F1F008F1863037
:10068000C1F030F18730A1F483E0809347010895F1
:100690008CEF92E0909344018093430181E080933A
:1006A000470182E58093450181E0809342010895EE
:1006B00080EC80934701089588E180934701089575
:1006C000823051F08330A1F780E380934701089591
:1006D0008CE080934701089580E680934701089558
:1006E0002CEF32E0309344012093430110924201F9
:1006F00091E090934701893059F070F08B3021F0F0
:100700008C3079F69093420181E5809345010895FC
:1007100082E5809345010895883019F683E580933A
:100720004501089526B59091470186B5821B89172A
:10073000E0F3089584B18C6284B92A982D9826B587
:100740009091470186B5821B8917E0F32A9A26B556
:100750009091470186B5821B8917E0F32A98809112
:100760004301909144018C5F924019F01092460130
:100770000895809145018CBD809142018DBD1092FC
:100780004601089584B1837D84B985B1837D85B99F
:100790001CBC0895CF93DF93C0E2E0914301F09138
:1007A00044018CEA0995E0914301F091440183E50D
:1007B0000995E0914301F091440180E00995D82F1B
:1007C000E0914301F091440180E00995D33561F156
:1007D0001CBC26B59091470186B5821B8917E0F3B2
:1007E0002A9A26B59091470186B5821B8917E0F3B6
:1007F0002A9826B59091470186B5821B8917E0F3A8
:1008000080914301909144018C5F924031F0C1503E
:1008100021F681E0DF91CF910895809145018CBD53
:10082000809142018DBDF3CF80E0DF91CF9108959B
:10083000CF92DF92EF92FF926B017C010E94020344
:100840008C2D880F880F880F8870E0914301F091FC
:10085000440180620995D701C60129E0B695A795A4
:10086000979587952A95D1F7E0914301F09144013E
:100870000995D701C601B695A79597958795E091FB
:100880004301F09144010995E0914301F091440145
:1008900080E0FF90EF90DF90CF900994CF92DF92AD
:1008A000EF92FF92CF93DF936B017C01C42FD22F85
:1008B0000E9402038C2D880F880F880F8870E091AA
:1008C0004301F091440180640995D701C60129E0F4
:1008D000B695A795979587952A95D1F7E09143010D
:1008E000F09144010995D701C601B695A795979552
:1008F0008795E0914301F09144010995E09143010E
:10090000F09144018C2F0995DD23E1F0CF37B9F048
:10091000D6B5CEE1C701B6010E9418048F3791F415
:1009200086B58D1B8D33B0F3D6B5C15099F781E0F4
:10093000DF91CF91FF90EF90DF90CF9008958FE0FF
:100940000E94430580E0DF91CF91FF90EF90DF9010
:10095000CF900895CF92DF92EF92FF92CF93DF93E3
:100960006B017C01C42F0E940203E0914301F091CE
:1009700044018CE40995D701C60129E0B695A795F5
:10098000979587952A95D1F7E0914301F09144011D
:100990000995D701C601B695A79597958795E091DA
:1009A0004301F09144010995E0914301F091440124
:1009B00080E00995CF3FF9F0D6B5CEE1C701B60189
:1009C0000E9418048F3F79F486B58D1B8D33B0F3E8
:1009D000D6B5C15099F781E0DF91CF91FF90EF90AC
:1009E000DF90CF90089580E0DF91CF91FF90EF905E
:1009F000DF90CF9008958FE00E94430580E0ECCF18
:100A0000CF93DF93EC01E0914301F091440180EA40
:100A10000995E0914301F09144018D2F0995E091F2
:100A20004301F09144018C2F0995E0914301F0912D
:100A3000440180E0DF91CF9109941F93CF93DF931E
:100A4000D82F192FC62FE0914301F091440180EC7B
:100A50000995E0914301F0914401812F0995E091BE
:100A60004301F09144018D2F0995E0914301F091EC
:100A700044018C2F09958EE10E94430580E0DF91AF
:100A8000CF911F910895882349F030E026B596B59F
:100A9000921B9C33E0F33F5F8313F8CF0895259AB0
:100AA00023982B9A50E217D05A95E9F70895AC0194
:100AB00088E605D0842F03D089E601D0852F0FD09A
:100AC00028E030E0382780FB869506D02A95D1F7BC
:100AD00030FB02D000D0689423982B9A16F02B9804
:100AE000239AE0914801F09149013197F0F72D9A4E
:100AF000E3B1E3FBE0914801F09149013197F0F750
:100B00002D98089520ECE7DF46F42A95E1F780E080
:100B10002AE1E5DF2A95E9F7DECF28E030E0DBDFE8
:100B2000869587F938272A95D1F7D5DF27F9322717
:100B300072F3D1DFD0CFDB01742FB9DF84E2BFDFE6
:100B4000E1DF8D937A95D1F70895DB01742FAFDF44
:100B500083EFB5DF8DE1B3DF84E6B1DF8D91AFDFE9
:100B600082E7ADDFCFDF8078D9F77A9589F70895EE
:100B7000CF93DF93EC018981813089F1823009F4D0
:100B8000A3C0833009F45DC08430B1F1873009F42B
:100B90007EC0853009F4F2C0863009F49AC08830EE
:100BA00009F4C9C0893009F4EFC08A3009F416C1CC
:100BB0008B3009F43EC18C3009F44FC18D3009F4FB
:100BC00066C18E3009F469C18F3009F4EEC08031FE
:100BD00009F40BC18F3709F421C180E029C0329B91
:100BE00052C080910E010E94320310920D01419873
:100BF0000E949A0380E01CC080910D0181110EC0FB
:100C00008A819B81092E000CAA0BBB0B80930901E2
:100C100090930A01A0930B01B0930C018E819F81E8
:100C2000909308018093070182E080930F018FEF7A
:100C300020E131E03093270120932601DF91CF910D
:100C40000895E0914301F09144018A8109958093D0
:100C50001001E0914301F09144018B81099580934B
:100C60001101E0914301F09144018C810995809339
:100C70001201E0914301F09144018D810995809327
:100C8000130184E0D5CF85E00E943203AECF80917E
:100C90000D0181110EC08A819B81092E000CAA0BC7
:100CA000BB0B8093090190930A01A0930B01B093B1
:100CB0000C018E819F81909308018093070183E04E
:100CC00080930F018FEFB4CF0E94C203419A80E05E
:100CD000AFCF80910D0181110EC08A819B81092EB9
:100CE000000CAA0BBB0B8093090190930A01A093FF
:100CF0000B01B0930C013C812D81822F8F7080936A
:100D0000040140E1249FC001112488279F70830FB4
:100D1000911D909306018093050120FD80930301AE
:100D20008E819F81909308018093070181E08093D9
:100D30000F018FEF7DCF80910D0181110EC08A814F
:100D40009B81092E000CAA0BBB0B80930901909389
:100D50000A01A0930B01B0930C01109206011092AE
:100D60000501109204018E819F8190930801809368
:100D7000070184E080930F018FEF5ACF0E94CA03CE
:100D80008093100181E054CF81E080930D018A812E
:100D90009B81AC81BD818093090190930A01A0934E
:100DA0000B01B0930C0180E043CF8A819B81092E17
:100DB000000CAA0BBB0B8093090190930A01A0932E
:100DC0000B01B0930C018E819F8190930801809359
:100DD000070185E080930F018FEF2ACF8A818093EE
:100DE0000E011092100181E023CF8A819B81092E90
:100DF000000CAA0BBB0B8093090190930A01A093EE
:100E00000B01B0930C018E819F8190930801809318
:100E1000070186E080930F018FEF0ACF81E0809376
:100E2000100110921101109212011092130184E02E
:100E3000FFCE8A819B8190934901809348012A9A31
:100E4000229A83E00E9443052A98419880E10E94FB
:100E500043050E944F0580E0EBCE80EC0E945F05C9
:100E600080E00E945F058AE00E9443052A9A85E09F
:100E70000E9443052A9885E00E94430584B1837D42
:100E800084B985B1837D85B9419A80E0D1CE0E9435
:100E900082058093100181E0CBCE8A810E945F059C
:100EA00080E0C6CEFF920F931F93CF93DF93582F0E
:100EB000792FF62E20910F013EEF320F323050F095
:100EC000253009F450C08FEFDF91CF911F910F9122
:100ED000FF9008956623B9F18091090190910A016C
:100EE000A0910B01B0910C01C52FD72F3FEF360F0A
:100EF0008E01030F111D1CC00E9400058883809184
:100F0000090190910A01A0910B01B0910C01019689
:100F1000A11DB11D8093090190930A01A0930B01BB
:100F2000B0930C01C017D10759F020910F01219601
:100F3000223011F7BC01CD010E9418048883DFCF55
:100F400087E08F1548F010920F018F2DDF91CF9120
:100F50001F910F91FF9008958F2DDF91CF911F91D9
:100F60000F91FF900895462F682F8091090190916D
:100F70000A010E949B058091090190910A01A091AC
:100F80000B01B0910C018F0D911DA11DB11D80931E
:100F9000090190930A01A0930B01B0930C018F2DCE
:100FA00093CFFF920F931F93CF93DF93382F792F17
:100FB000162F20910F01213071F0243061F026307E
:100FC00009F493C0FF24FA948F2DDF91CF911F91E4
:100FD0000F91FF900895112309F4B4C08091090185
:100FE00090910A01A0910B01B0910C01C32FD72F52
:100FF0001150AE01410F511D8A01F12C4FC02091BB
:10100000050130910601232B09F052C021E04881EF
:10101000BC01CD010E944E0480910701909108010E
:1010200001979093080180930701892BE9F41092AE
:101030000F018091040181FF38C08091030190E08D
:1010400020910501309106018217930771F160919B
:10105000090170910A0180910B0190910C01488166
:101060000E94AA04FF24F3948091090190910A013F
:10107000A0910B01B0910C010196A11DB11D8093AF
:10108000090190930A01A0930B01B0930C010C1776
:101090001D0709F499CF20910F012196213009F401
:1010A000AECF68810E941D05B7CFFF24F394DCCF3B
:1010B00020E04881BC01CD010E944E0480910301D3
:1010C0008150809303018111A7CF60910901709134
:1010D0000A0180910B0190910C0148810E94AA04A1
:1010E000809105018093030197CF462F682F80914F
:1010F000090190910A010E94A50580910901909132
:101100000A01A0910B01B0910C01810F911DA11D4D
:10111000B11D8093090190930A01A0930B01B09334
:101120000C018091070190910801811B9109909316
:10113000080180930701892B29F410920F01FF24E5
:10114000F39442CFF12C40CF1BB815B88BEF8AB97E
:101150008FEF84B914B883E087B99EEF98B985BD45
:101160000E94A90178940E947C00FDCFF894FFCFE3
:02117000FF5A24
:00000001FF
